:108000006C4300203DA3000055A3000057A30000CF
:1080100059A3000059A3000059A30000000000006C
:1080200000000000000000000000000059A3000054
:1080300059A300000000000059A30000A591000012
:1080400059A3000059A3000059A3000059A3000040
:1080500059A3000059A30000CB9D000059A30000C4
:1080600059A3000059A3000059A3000059A3000020
:1080700059A3000059A3000059A300001183000078
:1080800059A3000059A3000059A3000059A3000000
:1080900059A3000059A3000059A3000059A30000F0
:1080A00059A3000059A3000059A3000059A30000E0
:1080B00059A3000059A3000059A3000059A30000D0
:1080C00059A3000059A3000059A3000059A30000C0
:1080D00059A3000059A3000059A3000059A30000B0
:1080E00059A3000059A300000000000059A300009C
:1080F00059A3000059A3000059A3000059A3000090
:1081000059A3000059A30000F783000059A3000001
:10811000000000000000000059A3000059A3000067
:1081200059A3000059A3000059A3000059A300005F
:1081300059A3000059A3000059A3000059A300004F
:10814000000000000000000000000000000000002F
:1081500059A3000059A3000059A3000059A300002F
:10816000000000000000000000000000000000000F
:1081700000000000000000000000000000000000FF
:1081800000000000000000000000000000000000EF
:1081900000000000000000000000000000000000DF
:1081A00000000000000000000000000000000000CF
:1081B00059A3000059A3000059A3000059A30000CF
:1081C00059A3000059A3000059A3000059A30000BF
:1081D00059A3000059A3000059A3000059A30000AF
:1081E00059A3000059A3000059A30000000000009B
:1081F0000000000059A3000059A3000059A300008B
:1082000059A3000059A30000000000000000000076
:1082100059A3000059A3000059A3000059A300006E
:1082200059A3000059A3000059A3000059A300005E
:1082300059A3000059A3000059A3000059A300004E
:1082400059A3000059A3000059A3000059A300003E
:1082500059A3000059A3000059A3000059A300002E
:1082600059A3000059A3000059A3000070B52021B4
:10827000DFF8C00800F077FD0020DFF8BC180860C8
:108280002021DFF8B80800F06EFD0020DFF8B018FC
:10829000086000F0EEFA00F0A4FA00F073FB03238C
:1082A00006220121DFF89C0800F005FEDFF898683F
:1082B00040F21B303060DFF894484FF44770206084
:1082C00000F0AEFE050000F0ABFE401BB0F5FA7FFB
:1082D000F9D36420DFF8781809684143326891FBCC
:1082E000F2F1DFF870281160DFF86C18096800FB04
:1082F00001F0216890FBF1F0DFF8601808600520BC
:10830000DFF85C1808700120DFF85818086070BDAD
:1083100038B50220DFF850180860DFF8500802680E
:108320000168DFF84C381B689B0709D4DFF8443834
:108330001B689B0704D4DFF840381B68DB051BD49F
:10834000DFF80048216831F00201216000E0016897
:10835000DFF824180968C905F9D5DFF8E8570121C5
:10836000280000F013FE0121280000F015FE20680F
:1083700050F0020020603DE0DFF8004823680F2045
:1083800000FB0322102092FBF0F32360DFF8C027EC
:10839000DFF8C00700681B1ADFF8AC07006843432A
:1083A000642093FBF0F01060DFF8D4371C680F20D6
:1083B00000FB0411102091FBF0F11960DFF89837F1
:1083C000DFF898070068091ADFF880070068414362
:1083D000642091FBF0F01860DFF8A807006800281F
:1083E00004D41068DFF8A017086003E01868DFF80D
:1083F0009817086031BDDFF89407002101605FF431
:108400008021DFF88C271160FF22DFF888371A609F
:108410000160DFF88407016851F0020101607047D4
:10842000DFF874070068002801D1002000E0012077
:1084300070470120DFF8641708607047DFF82407F1
:108440000068002804D10020DFF8F416086003E07B
:108450002020DFF8EC16086070470020DFF8E016F7
:10846000086070472DE9F0410C00DFF8F816096844
:10847000002904D005002800C0B2072806DBDFF879
:108480001807016851F004010160A8E1DFF8D06627
:1084900028003178C0B2884200F0ED802800C0B2D8
:1084A000062803D13078022800F0E5802800C0B209
:1084B000022803D13078062800F0DD802800C0B201
:1084C000022803D02800C0B2062818D1DFF8D076E1
:1084D00000220321380000F0D6FE00220C213800D3
:1084E00000F0D1FE00F0C5F901220321380000F0B0
:1084F000CAFE01220C21380000F0C5FEA3E02800CE
:10850000C0B2052804D10020DFF82C1608609AE0DC
:108510002800C0B2002812D12020DFF81C16086005
:10852000DFF87C7600220321380000F0ACFE002248
:108530000C21380000F0A7FE00F09BF983E0280032
:10854000C0B201281CD1DFF8587600220321380080
:1085500000F099FE00220C21380000F094FE00F09B
:1085600088F901220221380000F08DFE0122082145
:10857000380000F088FE2020DFF8BC15086062E0BB
:108580002800C0B2042835D1DFF814760022032178
:10859000380000F078FE00220C21380000F073FE55
:1085A000DFF80076C021380000F0DDFB3021380014
:1085B00000F0D9FB00224021380000F0B7FB8022F8
:1085C0008021380000F0B2FB00221021380000F0BA
:1085D000ADFB20222021380000F0A8FB2020DFF88E
:1085E00058150860002300220121DFF8580500F02B
:1085F00062FC28E02800C0B203281ED100F039F93F
:10860000DFF89C754FF4FA624021380000F017FE45
:108610004FF4FA628221380000F011FE0321380085
:1086200000F02CFE01220321380000F02CFE012274
:108630000C21380000F027FE05E0DFF85C0501683A
:1086400051F0040101602800C0B2042803D02800C2
:10865000C0B2052807D1002300220121DFF8E4047D
:1086600000F029FC36E0002306220121DFF8D404C3
:1086700000F021FC2EE02800C0B2052821D1002006
:10868000DFF8B4140860DFF8187500220321380001
:1086900000F0F9FD00220C21380000F0F4FD00F09C
:1086A000E8F801220221380000F0EDFD0122082146
:1086B000380000F0E8FD0121DFF8880400F072FCCA
:1086C00008E02800C0B2042804D10121DFF87404B6
:1086D00000F068FC20002900C9B2022963D1DFF84C
:1086E000A484C8F80000D8F8004014F5FA64DFF854
:1086F000B07422004021380000F0A1FD2200822148
:10870000380000F09CFDD8F8000000280CD44FF48D
:1087100080724021380000F0E0FD4FF400724021EB
:10872000380000F0D4FD0BE04FF400724021380017
:1087300000F0D3FD4FF480724021380000F0C7FDF7
:108740000321380000F09AFDDFF83C040168642939
:1087500015DADFF854140968012910D100F060FC23
:10876000DFF848140968401A40F6B931884215D339
:10877000DFF82404016851F0010101600EE0006897
:1087800040F2F511884204DB0020DFF81C14086079
:1087900004E000F045FCDFF8141408600020DFF866
:1087A000101408601AE02900C9B2062902D100F0AD
:1087B0004FF913E000F034FCDFF8F01308600120FB
:1087C000DFF8E4130860DFF8D4030168012905D15C
:1087D0000021DFF8C4231160002101603570BDE87D
:1087E000F08110B5DFF8CC0300F0A0FDD14C0421DE
:1087F000200000F09FFA0221200000F09BFAD14CEB
:108800000021200000F003FC0720DFF8AC13086013
:108810001F2000F05DFF0121200000F035FB012149
:10882000200000F040FB002306220121200000F080
:1088300042FB012300220121200000F066FB62239D
:1088400001220121200000F060FB0121200000F046
:1088500025FB0121200000F01AFB1F2000F00CFF77
:108860000121200000F09EFB00211F2000F0F3FEFC
:1088700010BD38B5D14800F059FDD14800F09DFA3F
:10888000D04800F09AFAD04800F097FACF4800F0AC
:1088900094FAC44C4021200000F073FA802120009B
:1088A00000F06FFA1021200000F06BFA2021200068
:1088B00000F067FABA4CC64D2A004021200000F0B3
:1088C0009BFC2A008021200000F096FCE020C1499A
:1088D0000860B020C0490860AA20C04908604FF471
:1088E0007A624021200000F09DFC4FF47A628021E2
:1088F000200000F097FC4021200000F09DFC80212A
:10890000200000F099FC0321200000F0B9FC5FF486
:108910007020B349086000220F21200000F0C5FC40
:1089200001220F21200000F0C9FC00220F212000AD
:1089300000F0A9FC00220F21200000F0ADFC4FF454
:10894000FA624021200000F07AFC4FF4FA628221A2
:10895000200000F074FC0E230E224021200000F0C5
:1089600080FC0E230E228021200000F07AFC0321DF
:10897000200000F083FC4FF400724021200000F042
:10898000A6FC31BD70B56B4C0421200000F0D2F97B
:108990000221200000F0CEF9924C200000F0C6FC2D
:1089A000200000F0DDFC422000F092FE8E4C0221FF
:1089B000200000F069FA0221200000F074FA002182
:1089C000200000F024FB07208849086002212000D5
:1089D00000F00CFB40F6AC5540F6D86633002A0098
:1089E0000021200000F0FAFA33002A0001212000C3
:1089F00000F0F4FA41F61D552A000021200000F095
:108A0000E7FA2A000121200000F0E2FA20212000EC
:108A100000F0D6FA03230F220221200000F04BFAC7
:108A2000734B00220221200000F06FFA714B0122EB
:108A30000221200000F069FA0221200000F02EFA45
:108A4000422000F019FE0221200000F0D4FA70BD8F
:108A500070B50500564E280000F0E6FE30604A4C26
:108A600030682168884226DA6348006821688842B5
:108A700021D020683168411A4FF47A704143206850
:108A800091FBF0F13F4A106841434FF47A7091FB3B
:108A9000F0F01168081A1060106840F26D71884299
:108AA00003DB40F26C70106040E054481168814272
:108AB0003CDA10603AE020683168B1F5C87188424C
:108AC00008DB20683168884230DA4B48006821684A
:108AD00088422BD130682168411A4FF47A704143A3
:108AE000206891FBF0F1274E306841434FF47A70D3
:108AF00091FBF0F000F098FE0A2800DA0A20002D21
:108B000003D431684018306002E03168081A3060E0
:108B1000306840F26D71884203DB40F26C70306067
:108B200004E036483168814200DA3060206832491A
:108B3000086070BD0040024080400240007000406C
:108B40008070004000800340440300204803002060
:108B5000300300203C0300203403002040030020A9
:108B600068030020240300200C8003406880034039
:108B700010800340188003406C800340580300209D
:108B80005C0300204C0300203803002008900340C1
:108B90000C90034034900340200300202C0300205D
:108BA00000800240005000402803002054030020B1
:108BB00050030020003800F0C48F0340004000F054
:108BC00004180100041C0100041001000414010039
:108BD000BAAA050060800240A080024028800240BE
:108BE0001C800240013800F000900340C49F034005
:108BF00001000800220009006003002094F8FFFF34
:108C000030B5CB4300F58064D50725684CBF0D43D4
:108C10001D40256000F58460920747BF026811433C
:108C200001681940016030BDF0B5002400F6C4753C
:108C30000126A640314211D066002F684FF0030C88
:108C40000CFA06FC27EA0C072F60C2F34117D5F88F
:108C500000C007FA06F646EA0C062E60641C082CD3
:108C6000E6DBCC4300F5A065D6072E684CBF0E436B
:108C700026402E6000F2045596072E684CBF0E4326
:108C800026402E6000F5A16556072E684CBF0E43A6
:108C900026402E6000F5A36516072E684CBF0E43D4
:108CA00026402E6000F23C55D2062A684CBF0A438B
:108CB00022402A60DD0700F20C5215684CBF0D43BC
:108CC0002540156000F5A2629D0715684CBF0D4355
:108CD0002540156000F214525D0715684CBF0D4326
:108CE0002540156000F21C521D0715684CBF0D434E
:108CF0002540156000F244529D0515684CBF0D4398
:108D00002540156000F5A86213F4407F156814BF74
:108D10000D432540156000F5A560002B07BF0268D4
:108D200041EA020401680C400460F0BD00EB8100E0
:108D30000260704738B5FFE704460D460022FFF792
:108D40005FFF2946204601B0BDE8304000230122E4
:108D50006AE738B500F02DF82946204601B0BDE895
:108D600030400823F3E738B504460D460823FFE7F3
:108D70000122FFF759FF29462046BDE8384001226D
:108D80003EE738B500F007F82946204601B0BDE8B7
:108D900030400823DBE704460D46022230E738B5B1
:108DA000FFF7F9FF2946204601B0BDE8304008230F
:108DB000CDE704460D46002222E710B50D4B0FF219
:108DC00038021C68C0F30741CC40E40746BF02EB01
:108DD000C101496852F8311001F22C51020A0B68A6
:108DE0000F24944000F00F00A34390401843086004
:108DF00010BD00006CE00F400040004000800540C6
:108E000000500040009005400060004000A0054078
:108E10000070004000B005400040024000C0054026
:108E20000050024000D005400060024000E00540D4
:108E30000070024000F0054000D0034000000640F2
:108E400000100640001006400020064000200640AA
:108E5000003006400030064000400640004006401A
:108E6000005006400050064000600640006006408A
:108E700000700640007006400080064000800640FA
:108E8000009006400090064050F8082F0CE00122A8
:108E900002FA01F100F10C021160B3E00268012353
:108EA00003FA01F1B0E00268012303FA01F122EABA
:108EB000010101607047F0B500F1140689000F252B
:108EC0008D403468ED4302F00F0705EA040C07FA01
:108ED00001F444EA0C04346003F0030300F12004BD
:108EE00003FA01F126683540BF1F2943032F216093
:108EF0000AD8FF0050F81C1F3023BB4002F030029C
:108F00009943BA400A430260F0BD70B5490140314F
:108F1000081892000F2191400468C94303F00F051F
:108F20000C4095402C430460C3F3032600F1180461
:108F3000964025680D4035432560041DC3F3031694
:108F400000F01EF800F11C04C3F3035600F018F8FB
:108F50000124944013F4702F00F110050BD050F849
:108F6000146FC3F30243314003FA02F20A43026072
:108F70002868044302E0286820EA04042C6070BDDD
:108F800025680D409640354325607047012202FA5E
:108F900001F140F8101F7047012202FA01F140F878
:108FA000181F704710B50B0C012401F00F0150F889
:108FB000282F04FA01F141EA03411143016010BD79
:108FC000002200E0521C4908FCD140F8302F7047C5
:108FD00000EB810000F560600260704700EB8100EB
:108FE00000F5646042EA03420260704750F8082FBF
:108FF0004FF4803359E750F8082F4FF4803303FAC9
:1090000001F101E050F8082F11430160704750F85A
:10901000382F920841EA820101607047872070472B
:1090200063480068704738B500F00EFB4FF400400D
:109030006049086000F01AFC5F4800F09FF90120C9
:1090400000F098F95D4C200000F070F95C4800F0E9
:109050006DF95C4D280000F069F95B4800F066F995
:109060005A4800F063F95A4800F060F9594800F096
:109070005DF900F033FC200000F074FA280000F0E5
:1090800071FA554800F0C4FC00F0B6FC00210F2036
:1090900000F0E1FA0F2000F0EFFA00F0B3FC00F06E
:1090A000CFFA4E4800F042F900F0BAFC4C4800F00C
:1090B000CCFC4C4C10212000FFF755FE0823662203
:1090C00010212000FFF7B0FD002047490860474C01
:1090D00040221021200000F01EFC206845280BD102
:1090E0006068312808D1A068342805D1E0683028AC
:1090F00002D12069302802D0102000F04AFD04225D
:109100000421684600F007FC9DF80000342803D1D4
:109110009DF8010031280CD034208DF8000031205A
:109120008DF8010004220421684600F009FC0028A3
:10913000F8D15FF0704000F0F9F85FF0804000F087
:1091400049FD012803D15FF0804000F03BFD284934
:109150005FF0804000F045FD5FF0804000F027FDAB
:109160005FF0804000F045FD5FF0804000F01EFDA4
:109170005FF0804000F021FD31BD80B55FF08040A0
:1091800000F028FD012803D15FF0804000F01AFDB7
:1091900018495FF0804000F024FD5FF0804000F04F
:1091A0000CFD01BD02480168491C016070470000C8
:1091B0006403002008ED00E0800300C1000800F017
:1091C000010800F0020800F0030800F0040800F0B5
:1091D000050800F0005800F080380100000C00F095
:1091E0000000002000500240405002404802002091
:1091F00000B4C40400350C00401801686FF352013C
:109200001143016000F124012030920704D5B022FF
:1092100002604FF4306003E08C22026040F60C00E4
:1092200008607047401800F11001006883074CBFC8
:109230005208521E0A607047081801681AE010B5FB
:109240008B0900EB831003689C0700F1100348BFF3
:1092500052081B689A1AC9074CBF1C3018300260AC
:1092600010BD401800F12C010A6000F130010B60C4
:1092700050F8281F41F001010160704701607047FC
:1092800040F8041F70470830012A02680CBF1143E0
:1092900022EA0101016070470C30012A02680CBF0C
:1092A000114322EA0101016070472430012A02685B
:1092B0000CBF114322EA0101016070471030012AFE
:1092C00002680CBF114322EA0101016070470818CF
:1092D00050F8041F0A4302607047081850F8041F32
:1092E00021EA02020260704718B58100DFF88C2283
:1092F000C0F3072301F47F71D31841EA431343F00D
:10930000844301241C600023009302E0009C641C41
:109310000094009B102BF9D3C0F30720121841EAE8
:10932000421141F084410020086011BDC0F30722C2
:10933000DFF84C1280008A1800F47F7040EA421077
:1093400040F0844001210160704780008A1800F4D9
:109350007F7040EA421040F0844000210160704775
:10936000C0F30722DFF81C12EFE700000138FDD13F
:1093700070477047DFF814120860704770B5DFF867
:1093800008221369146A014623F4800301F00105E1
:1093900043F4006303F0010085F0010544F4006428
:1093A0001361284214620ED061F0010003404FF4B3
:1093B0008070906013614FF400201568EE054AD468
:1093C000401EFAD170BD080960F30A13DFF8CC0122
:1093D00013610440DFF8C80108400443C80000F0EE
:1093E000400004431462480B60F34D3360F34D3486
:1093F00040209060002C47BF146213611361146217
:10940000DFF8A0010340DFF8A00108400343C80DC6
:1094100060F3DC54480008D5DFF8900124F48004A0
:10942000084043F48003044301E024F0804408052D
:109430000BD44FF400405E490D68EE0701D4401E86
:10944000FAD123F4006324F4006413611462102041
:10945000BDE870408AE70028B5D170BDF0B5554928
:109460000A6D0B6E002B4CBF03F0700002F0300051
:1094700040B1102847D0202847D0302847D0702846
:1094800048D04AE00FF24C10C2F3841450F8245034
:10949000494C04EA0306B6F1004F4FF0FF3003D009
:1094A000002B41D416053FD43A4E376876680968D8
:1094B000C6F3042C06F01F060CF1010C761C16FBFB
:1094C0000CF67600B5FBF6F5C7F30906C7F3892756
:1094D0006F4301F47041BF0AB1F5005F06FB0575EB
:1094E00042F480020DD0B1F5405F18D0B1F5804F45
:1094F00017D0B1F5E04F16D0B1F5104F08BF2F4887
:1095000012E02F4810E0224DC2E72E4DC0E747F28F
:109510003055BDE74FF40045BAE70020F0BD2A48BA
:1095200002E02A4800E01C48510217D5002B10D554
:1095300059000BD51C40B4F1004F03D0002B05D4CB
:10954000110503D46D00C3F3865104E0C3F3C55184
:1095500001E0C2F3C351491CB5FBF1F5A84288BF35
:109560002846F0BD1A4901230A6800F00F0003FAEB
:1095700000F000E00A6810430860704700E50F4003
:1095800000E60F4000E80F4050E00F407CE00F4045
:109590000024F40060E10F4040787D018FFFFF7FE1
:1095A00030000080FEFF3FF80100C007000040408F
:1095B00068E10F4010E00F4000080080002D3101ED
:1095C00000B4C40400093D0080F0FA02005A6202AF
:1095D0006CE00F4040420F0000201C0080841E0001
:1095E00000802500999E36000040380000093D00AB
:1095F00000803E0000004B00404B4C0000204E001D
:10960000808D5B0000C05D000080700000127A0059
:1096100000007D0080969800001BB7000080BB0012
:10962000C0E8CE00647ADA000024F4000000FA00FA
:1096300080A81201002D310100366E0140787D01B5
:1096400080B500F0E1FA02E080B500F0D9FA00B18F
:109650000120C0B202BD10B50FF2D402830852F847
:1096600023201368C00000F01800FF248440A343A7
:1096700081401943116010BD04282B4903D10868AB
:1096800040F480300BE0052804D10A6842F400322F
:109690000A607047062804D1086840F480200860FA
:1096A00070470F2805D12148016841F0020101608F
:1096B00070470CD90FF21413A0F1100110384009B3
:1096C00053F82000012201F01F018A400260704718
:1096D0000428154903D1086820F480300BE00528E0
:1096E00004D10A6822F400320A607047062804D1C7
:1096F000086820F48020086070470F2805D10B48C7
:10970000016821F00201016070470CD90FF2D0030B
:10971000A0F110011038400953F82000012201F097
:109720001F018A400260704724ED00E010E000E075
:109730000000000018ED00E01CED00E020ED00E06E
:1097400000E400E004E400E008E400E00CE400E0F1
:1097500010E400E014E400E018E400E01CE400E0A1
:1097600020E400E024E400E028E400E02CE400E051
:1097700030E400E034E400E038E400E03CE400E001
:1097800040E400E044E400E048E400E04CE400E0B1
:1097900050E400E054E400E058E400E05CE400E061
:1097A00060E400E064E400E068E400E06CE400E011
:1097B00070E400E074E400E078E400E07CE400E0C1
:1097C00080E400E084E400E088E400E000E100E000
:1097D00004E100E008E100E00CE100E010E100E05D
:1097E00080E100E084E100E088E100E08CE100E05D
:1097F00090E100E000210100C9B230390A2902D20B
:109800003038C0B208E00100C9B24139062902D29D
:109810003738C0B200E00020704710F00F00014957
:10982000085C7047B0A30000002801D54042FFE764
:10983000704730B4002513E050F8042BD30744BF21
:10984000A9F101039A18091F042942F8045BFAD20E
:1098500013468C0744BF15809B1CC90748BF1D7069
:1098600050F8041B0029E7D130BC7047024801685A
:1098700041F040410160704734EF00E038B50446E4
:1098800000F029F8544D0321296000F024F801204C
:10989000E40900FA04F45148E443046000F01BF8C2
:1098A000002028600A20BDE83240FFF75FBD10B5F8
:1098B00000F011F8484C0321216000F00CF84749F2
:1098C0000020086000F007F8002020600A20BDE8B2
:1098D0001040FFF74BBD0A20FFF748BD10B502202E
:1098E000FFF744FD3E4C2168C807FCD4606810F0C7
:1098F0000C0F0CD13B48FFF7F7FC0220FFF736FDB9
:109900002068C107FCD4606810F00C0F01D0022061
:1099100010BD002010BD10B5334B8C091C60C1F385
:109920008301920859600AD004E0596811B91C6893
:10993000641C1C60521E196940F8041BF5D110BD4F
:109940002DE9F84F81468A46274D6869C007FCD447
:10995000DFF89880264F274E4FEA9A102860940827
:10996000CAF38300686005D12AE0686810B92968E5
:10997000491C296030683840404505D130680104F1
:1099800004BF5046FFF77AFFD9F800002861FFF7BF
:10999000A2FFD5F814B05FEACB70FAD45FEACB60CF
:1099A0000AD530680740474504D13068010408BF34
:1099B000FFF77DFF58460DE0641E09F10409D4D17C
:1099C00030680740474504D13068010408BFFFF7FD
:1099D0006EFF6869BDE8F28FFCD00F40C0E20A401C
:1099E00018F00A40005800F004F00A40000005108A
:1099F0000000FF7000E00F400748016841F00501DA
:109A0000016070470448016841F00201016070473D
:109A10000249401E0860704710E000E014E000E0DA
:109A20004C49FFE7012008607047012100F01F004A
:109A300001FA00F0484908607047012100F01F005A
:109A400001FA00F0454908607047454908607047D1
:109A500000F01F00012202FA00F0424ACB0748BF83
:109A600010608B0748BF90614B0748BF1062090721
:109A700048BF906070473A4A126800F03F0002EB1E
:109A80000012394893680340194391607047F0B55C
:109A9000334C2568354C00F03F0005EB0016B768E5
:109AA0002740840604D5042914BF062941F001018A
:109AB000DDF814C0ACF1010E41EA0E14274307F0A3
:109AC0004064B4F1406F04D0A40E0CFA04F4A21860
:109AD000521E326007F04042B2F1404F0FD00429CD
:109AE00018BF062906D140F0200005EB001000F158
:109AF0000C0304E0920F0CFA02F003445B1E736047
:109B0000B760F0BD1649096800F03F0001EB001096
:109B1000806800F007004108490004291EBF420880
:109B20005200062A04BF40084000704700F0FF01C1
:109B300010B5CB080E4A02EB8302890001F01C012C
:109B400013680F248C40000CA34388401843106016
:109B500010BD000004F00F4028F00F402CF00F4023
:109B600008F00F401CF00F40F73FFC0008C0FFFF5B
:109B700010F50F4080B50C4A1368010089B28B4381
:109B800013604FF6FF7180B2884201D1FEF751FC9D
:109B900001BD05490A6880B2104308607047024958
:109BA000096880B208407047000300201BE050F8AD
:109BB000081F41F002010160704700F5406001217B
:109BC0000160704700F54060014901607047000086
:109BD00051E5CC1A00F540600068012818BF00204C
:109BE00070470160704750F8081F41F001010160A3
:109BF000704700F58360016841F48071016070472F
:109C0000EFF3108072B67047EFF3108062B67047C2
:109C100010B5DFF84404FFF789FBDFF84004FFF7D5
:109C2000CCF8DFF83C04FFF7C8F83021DFF8340443
:109C3000FFF7B5F8FFF712FCDFF82C4460235FF460
:109C4000E1320100200000F041FA10220221200040
:109C500000F038FADFF81404016831F010010160F7
:109C60001021200000F085FA200000F05EFA0321A8
:109C7000200000F08CFA1620FFF758FF1720FFF79E
:109C800055FFC0211620FFF7E6FC1620FFF7F4FC75
:109C90000F211620FFF7DCFEDFF8D4131620FFF7A4
:109CA000EAFE0F211720FFF7D3FEDFF8C8131720B5
:109CB000FFF7E1FE4FF40070FFF76BFF4FF4807089
:109CC000FFF767FF00F063F9FFF7AAF9DFF8A813C1
:109CD00008600120DFF8A413086010BD38B5DFF874
:109CE0009C03006800286FD0FFF79AF9DFF88843DB
:109CF0002168401A652807D34FF48070FFF749FFA9
:109D000000210520FEF7AEFB00F0C9F8C0B2012823
:109D10005AD1DFF86C536878BB2805D1DFF86403AB
:109D2000DFF864130860F9E7A878C0281FD1FFF7AF
:109D300077F920604FF48070FFF71CFFE9782879ED
:109D400070F0FF00042907D1C043002804D04FF46D
:109D50000070FFF70FFF03E04FF40070FFF719FFEB
:109D600000F050F800210520FEF77CFB2CE0C12814
:109D70002AD12979687951EA0021A87951EA00416C
:109D8000E87951EA0061E878FEF76CFB2D7AE80784
:109D900002D4FEF762FB01E0FEF750FBFFF740F94B
:109DA00020604FF48070FFF7E5FEA80703D5B548A3
:109DB000B5490860FBE7680703D54FF6FF70FFF76A
:109DC000D9FE012000F038F831BD10B5A64C0121B4
:109DD000200000F0D3F90100200000F0D5F9AB48D5
:109DE0000068002807D11620FFF78CFE002808D154
:109DF00000F0CDF805E0A6480068800601D500F027
:109E0000C6F810BD10B5A34C05202070002060706E
:109E1000C020A070FFF702F9E070E078C043207125
:109E2000342060713120A0719B4C00F0DAF8206082
:109E3000206800F0C7F810BD10B5964C08212170BD
:109E400000216170C221A170012802D10020E070C0
:109E500001E0FF20E070FEF7E3FA012803D10220C1
:109E6000FFF797FE02E00220FFF784FE4FF6FF7037
:109E7000FFF795FE20710100090A61710100090CCC
:109E8000A171000EE0710020207200206072824CEF
:109E900000F0A7F82060206800F094F810BD2DE9CC
:109EA000F843002000E0401C642806DA7B490A5C85
:109EB000032AF8D1040000220A54642801DB0020A0
:109EC00063E0671E00E07F1E002F5DD4734DE85DE8
:109ED0000228F8D10020E855E41B641C083CE00788
:109EE00001D5022051E06408201F2F2801D3022051
:109EF0004BE0781C00F0FF00411C01F0FF01604EB8
:109F0000695C285C00F0CEF830703078844201D073
:109F100002203AE05FF00108F81C00F0FF00411C4D
:109F200001F0FF01695C285C00F0BCF8707070788B
:109F300018EB00085FF0000917E0781D10EB4900EE
:109F400000F0FF00411C01F0FF01695C285C00F09B
:109F5000A9F806EB09018870A14504D206EB0900B7
:109F6000807858FA80F819F101094C45E5D27FEA6A
:109F7000080808F0FF0806EB04008078804501D04F
:109F8000022002E0012000E00020BDE8F28380B55D
:109F900000203E4908601620FFF74FFD002003E037
:109FA00000213E4A1154401C6428F9D364200090DB
:109FB0003A4B2D4A01211620FFF769FD1620FFF7C5
:109FC00034FD01BD80B50121304A11600090264B5F
:109FD000334A01211720FFF75AFD1720FFF725FD0F
:109FE00001BDF8B501262E4D02202870002415E091
:109FF000385DC0B20009C0B2FFF70FFC05EB4401A9
:10A000004870385D10F00F00FFF707FC05EB4401C6
:10A010008870002C01D0385D3618641C1D4F3878CC
:10A02000401CA042E4D2F64306F0FF0630000009CF
:10A03000FFF7F3FB05EB4401487016F00F06300004
:10A04000FFF7EBFB05EB44018870032005EB4401AF
:10A05000C8706000001DF2BD011800F0021002007F
:10A060000214020000A0054000D000402CD00040A7
:10A070000080000C008000C00C03002004030020BE
:10A08000880200200400FA050CED00E01003002017
:10A090003CD00040BC0200200803002080010020CA
:10A0A000E401002038B50C000021C0B2FFF7A2FB8C
:10A0B00005002D012000C0B2FFF79CFB45192800C8
:10A0C000C0B232BD114340F8341F7047F8B50446A2
:10A0D0000E4617461D4600F035F8B6EB071F04F193
:10A0E000300005D2016841F0200101607F0803E0E3
:10A0F000026822F020020260F600B6FBF7F0401C76
:10A10000400804F124028109116000F03F0004F1CD
:10A110002801086004F12C0004F1180105600020FA
:10A1200008602046BDE8F240FFE700F12C010A6814
:10A1300042F010020A6040F2013150F8303F0B4308
:10A140000360704700F118010A681307FCD400F19E
:10A150002C010A6822F010020A6050F8303F0249D0
:10A160000B40036070470000FEFCFFFF11430160DD
:10A17000704750F8302F22F01002F7E7002914BF83
:10A1800040303C300068704740F8441F704750F83A
:10A19000482FEBE780B500202649086010212648AB
:10A1A000FEF7D7FD02212548FEF7DDFD00202449FA
:10A1B000086040212348FEF7D6FD002022490860B0
:10A1C000FEF72EFF2149086001202149086001BDEA
:10A1D00010B51F48006800282AD0FEF721FF1B4950
:10A1E0000968401A0A2823D300211A480068002869
:10A1F00001D051F001010F4C0422174800F032F851
:10A2000020602078C00703D5144815490860FBE793
:10A2100040200D4908604FF6FF70FFF7C0FC002892
:10A2200003D002200649086002E0002004490860CB
:10A2300010BD0000180300200080054000500240BF
:10A240000850024000A0054000A105401C0300206A
:10A250001403002040800540F00200200400FA05AD
:10A260000CED00E070B40B00002503E050F8254031
:10A2700023436D1C541EA542F8D300EB820454F80E
:10A28000044C23400D00002603E050F826402540F2
:10A29000761C541EA642F8D32B4300EB820444F8EC
:10A2A000043C921E06E000EB820454F8044C40F893
:10A2B0002240521E002AF6D10160180070BC70477F
:10A2C00010B5074979441831064C7C44163404E033
:10A2D0000A68081D114488470146A142F8D110BD03
:10A2E0002C000000380000004EF68851CEF200012C
:10A2F000086840F470000860BFF34F8FBFF36F8FA2
:10A300004FF00070E1EE100A7047000027F5FFFFE4
:10A310006C030000000000200000000080B5FEF784
:10A3200082FEFFF737FFFDF7A1FFFFF771FCFEF795
:10A3300024FFFFF74DFFFFF7D1FCF8E780B5044895
:10A34000016851F47001016000F008F801BD0000DF
:10A3500088ED00E0FEE7FEE700BFFDE7AFF3008019
:10A36000FFF7C2FF00F000F800F00DF8002801D060
:10A37000FFF7A6FFAFF300800020AFF30080FFF7E8
:10A38000CDFF00F002F80120704700F001B8000096
:10A390000746384600F002F8FBE7000080B5AFF34F
:10A3A0000080024A11001820ABBEFBE72600020025
:10A3B00030313233343536373839414243444546FB
:040000050000A35DF7
:00000001FF
